 adc

 Timestamp is 4fb04cb0 (Mon May 14 12:07:12 2012)

 Preferred load address is 10000000

 Start         Length     Name                   Class
 0001:00000000 00000004H .CRT$XCA                CODE
 0001:00000004 00000004H .CRT$XCZ                CODE
 0001:00000008 00000004H .CRT$XIA                CODE
 0001:0000000c 00000004H .CRT$XIZ                CODE
 0001:00000010 00000004H .CRT$XPA                CODE
 0001:00000014 00000004H .CRT$XPZ                CODE
 0001:00000018 00000004H .CRT$XTA                CODE
 0001:0000001c 00000004H .CRT$XTZ                CODE
 0001:00000020 000000b0H .rdata                  CODE
 0001:000000d0 00000020H .rdata$debug            CODE
 0001:000000f0 00000df0H .text                   CODE
 0001:00000ee0 00000048H .xdata                  CODE
 0001:00000f28 0000003cH .idata$2                CODE
 0001:00000f64 00000014H .idata$3                CODE
 0001:00000f78 00000060H .idata$4                CODE
 0001:00000fd8 0000004cH .idata$6                CODE
 0001:00001030 00000106H .edata                  CODE
 0002:00000000 00000060H .idata$5                DATA
 0002:00000060 00000008H .data                   DATA
 0002:00000068 00000014H .bss                    DATA
 0003:00000000 000000e0H .pdata                  DATA

  Address         Publics by Value              Rva+Base       Lib:Object

 0000:00000000       ___safe_se_handler_count   00000000     <absolute>
 0000:00000000       ___safe_se_handler_table   00000000     <absolute>
 0001:00000000       __xc_a                     10001000     corelib0:crt0init.obj
 0001:00000004       __xc_z                     10001004     corelib0:crt0init.obj
 0001:00000008       __xi_a                     10001008     corelib0:crt0init.obj
 0001:0000000c       __xi_z                     1000100c     corelib0:crt0init.obj
 0001:00000010       __xp_a                     10001010     corelib0:crt0init.obj
 0001:00000014       __xp_z                     10001014     corelib0:crt0init.obj
 0001:00000018       __xt_a                     10001018     corelib0:crt0init.obj
 0001:0000001c       __xt_z                     1000101c     corelib0:crt0init.obj
 0001:000000f0       BSPADCCIomuxConfig         100010f0 f   adc.obj
 0001:000000f8       BSPADCEnableClock          100010f8 f   adc.obj
 0001:00000118       BSPADCGetIPGClock          10001118 f   adc.obj
 0001:0000013c       BSPADCGetHSYNCPolarity     1000113c f   adc.obj
 0001:00000144       BSPADCGetHSYNCEnable       10001144 f   adc.obj
 0001:0000014c       ADC_Deinit                 1000114c f   adc_common_topaz_v1:adc.obj
 0001:00000188       ADC_Init                   10001188 f   adc_common_topaz_v1:adc.obj
 0001:000002a8       ADC_Open                   100012a8 f   adc_common_topaz_v1:adc.obj
 0001:000002cc       ADC_Close                  100012cc f   adc_common_topaz_v1:adc.obj
 0001:000002ec       ADC_IOControl              100012ec f   adc_common_topaz_v1:adc.obj
 0001:00000a3c       ADC_Read                   10001a3c f   adc_common_topaz_v1:adc.obj
 0001:00000a44       ADC_Write                  10001a44 f   adc_common_topaz_v1:adc.obj
 0001:00000a4c       ADC_Seek                   10001a4c f   adc_common_topaz_v1:adc.obj
 0001:00000a54       ADC_PowerUp                10001a54 f   adc_common_topaz_v1:adc.obj
 0001:00000a58       ADC_PowerDown              10001a58 f   adc_common_topaz_v1:adc.obj
 0001:00000a5c       LocalFree                  10001a5c f   coredll:COREDLL.dll
 0001:00000a6c       DeleteCriticalSection      10001a6c f   coredll:COREDLL.dll
 0001:00000a7c       Sleep                      10001a7c f   coredll:COREDLL.dll
 0001:00000a8c       InitializeCriticalSection  10001a8c f   coredll:COREDLL.dll
 0001:00000a9c       LocalAlloc                 10001a9c f   coredll:COREDLL.dll
 0001:00000aac       GetTickCount               10001aac f   coredll:COREDLL.dll
 0001:00000abc       LeaveCriticalSection       10001abc f   coredll:COREDLL.dll
 0001:00000acc       EnterCriticalSection       10001acc f   coredll:COREDLL.dll
 0001:00000adc       SetLastError               10001adc f   coredll:COREDLL.dll
 0001:00000aec       MmUnmapIoSpace             10001aec f   ceddk:CEDDK.dll
 0001:00000afc       MmMapIoSpace               10001afc f   ceddk:CEDDK.dll
 0001:00000b0c       DDKClockSetGatingMode      10001b0c f   cspddk:CSPDDK.dll
 0001:00000b1c       DDKClockGetFreq            10001b1c f   cspddk:CSPDDK.dll
 0001:00000b2c       DllMain                    10001b2c f   corelib0:dllmain.obj
 0001:00000c48       _DllMainCRTStartup         10001c48 f   corelib0:pegdmain.obj
 0001:00000d74       _cexit                     10001d74 f   corelib0:cexit.obj
 0001:00000d90       _initterm                  10001d90 f   corelib0:crt0dat.obj
 0001:00000dc4       _cinit                     10001dc4 f   corelib0:crt0dat.obj
 0001:00000df8       __security_init_cookie     10001df8 f   corelib0:seccinit.obj
 0001:00000e54       __C_specific_handler       10001e54 f   corelib1:COREDLL.dll
 0001:00000e64       memset                     10001e64 f   corelib1:COREDLL.dll
 0001:00000e74       _XcptFilter                10001e74 f   corelib1:COREDLL.dll
 0001:00000e84       free                       10001e84 f   corelib1:COREDLL.dll
 0001:00000e94       __security_gen_cookie2     10001e94 f   corelib1:COREDLL.dll
 0001:00000ea4       CspADCTouchGetBaseRegAddr  10001ea4 f   adc_mx25_topaz_v1:adc.obj
 0001:00000eb0       DisableThreadLibraryCalls  10001eb0 f   coredll:COREDLL.dll
 0001:00000ec0       InterlockedExchange        10001ec0 f   coredll:COREDLL.dll
 0001:00000ed0       TerminateProcess           10001ed0 f   coredll:COREDLL.dll
 0001:00000f28       __IMPORT_DESCRIPTOR_COREDLL 10001f28     coredll:COREDLL.dll
 0001:00000f3c       __IMPORT_DESCRIPTOR_CEDDK  10001f3c     ceddk:CEDDK.dll
 0001:00000f50       __IMPORT_DESCRIPTOR_CSPDDK 10001f50     cspddk:CSPDDK.dll
 0001:00000f64       __NULL_IMPORT_DESCRIPTOR   10001f64     coredll:COREDLL.dll
 0002:00000000       __imp_MmUnmapIoSpace       10003000     ceddk:CEDDK.dll
 0002:00000004       __imp_MmMapIoSpace         10003004     ceddk:CEDDK.dll
 0002:00000008       \177CEDDK_NULL_THUNK_DATA  10003008     ceddk:CEDDK.dll
 0002:0000000c       __imp_InitializeCriticalSection 1000300c     coredll:COREDLL.dll
 0002:00000010       __imp_LocalAlloc           10003010     coredll:COREDLL.dll
 0002:00000014       __imp_GetTickCount         10003014     coredll:COREDLL.dll
 0002:00000018       __imp_Sleep                10003018     coredll:COREDLL.dll
 0002:0000001c       __imp_EnterCriticalSection 1000301c     coredll:COREDLL.dll
 0002:00000020       __imp_SetLastError         10003020     coredll:COREDLL.dll
 0002:00000024       __imp_DeleteCriticalSection 10003024     coredll:COREDLL.dll
 0002:00000028       __imp_LeaveCriticalSection 10003028     coredll:COREDLL.dll
 0002:0000002c       __imp_LocalFree            1000302c     coredll:COREDLL.dll
 0002:00000030       __imp_TerminateProcess     10003030     coredll:COREDLL.dll
 0002:00000034       __imp_InterlockedExchange  10003034     coredll:COREDLL.dll
 0002:00000038       __imp___C_specific_handler 10003038     corelib1:COREDLL.dll
 0002:0000003c       __imp_memset               1000303c     corelib1:COREDLL.dll
 0002:00000040       __imp__XcptFilter          10003040     corelib1:COREDLL.dll
 0002:00000044       __imp_free                 10003044     corelib1:COREDLL.dll
 0002:00000048       __imp___security_gen_cookie2 10003048     corelib1:COREDLL.dll
 0002:0000004c       __imp_DisableThreadLibraryCalls 1000304c     coredll:COREDLL.dll
 0002:00000050       \177COREDLL_NULL_THUNK_DATA 10003050     coredll:COREDLL.dll
 0002:00000054       __imp_DDKClockSetGatingMode 10003054     cspddk:CSPDDK.dll
 0002:00000058       __imp_DDKClockGetFreq      10003058     cspddk:CSPDDK.dll
 0002:0000005c       \177CSPDDK_NULL_THUNK_DATA 1000305c     cspddk:CSPDDK.dll
 0002:00000060       __security_cookie          10003060     corelib0:seccinit.obj
 0002:00000064       __security_cookie_complement 10003064     corelib0:seccinit.obj
 0002:00000068       _exitflag                  10003068     corelib0:cexit.obj
 0002:0000006c       __onexitend                1000306c     <common>
 0002:00000070       __onexitbegin              10003070     <common>
 0002:00000074       g_pcsExit                  10003074     <common>
 0002:00000078       _pRawDllMain               10003078     <common>

 entry point at        0001:00000c48

 Static symbols

 0001:00000b4c       _DllMainCRTStartupHelper   10001b4c f   corelib0:pegdmain.obj
 0001:00000c78       doexit                     10001c78 f   corelib0:cexit.obj
